:020000040000FA
:06080000A6EF24F0120037
:060808002CEF17F01200B6
:02080E00C250D6
:08081000020B01E0010E1200D1
:0608180033EF1DF0120099
:02081E000400D4
:10082000024A0000C707000028000000D449000069
:10083000990700002E000000D0490000EF070000DB
:1008400004000000AC490000000300002400000088
:0C08D4008E0E376E3D6A346A336A7EEF88
:1008E00004F08E0E376E36C03DF0346A336A36AE91
:1008F0007EEF04F0356C361EE86A3622426AE86AFA
:100900003664A7EF04F0F00E3614E86690EF04F0BA
:10091000363A35380F0B36263538F00B356E4284B3
:10092000D89036BEA3EF04F035363636422A36BEAE
:10093000A3EF04F035363636422A36BEA3EF04F074
:1009400035363636422A4250375E15EF05F035C04F
:1009500036F0356AE86A428636640FEF05F0F00E2D
:100960003614E866B6EF04F0363A4284D89036BEC4
:10097000A3EF04F03636422A36BEA3EF04F0363633
:10098000422A36BEA3EF04F03636422AA3EF04F023
:100990003E803EAEFF0C366A3DAE366836C035F05E
:1009A00036C034F036C033F03D363632FF0C3E8070
:1009B0003EAEFF0C366A3DAE366836C035F036C006
:1009C00034F03D363632FF0C3E803EAEFF0C366AC8
:1009D0003DAE366836C035F03D363632FF0C3E80CF
:1009E0003EAEFF0C366A3DAE36683D363632FF0C01
:1009F0003E823EAEFF0C37683668356834683D3657
:100A00003632FF0C3E843EAEFF0C010E376E366A66
:100A1000356A346A3D363632FF0C3E86FF0C366A44
:100A2000356A346A336A376A000C3DAE369E000C74
:100A30009E0E376E3D6A2CEF05F09E0E376E36C067
:100A40003DF036AE2CEF05F0E86A336C341E351EEF
:100A5000361E3422352236223650FF0BD8B491EFA1
:100A600005F0F00BD8B46AEF05F0E86A36BE53EF34
:100A700005F0D8903336343635363636E82A36BE69
:100A80004FEF05F03336343635363636E82A36BE83
:100A90004FEF05F03336343635363636E82A3764CC
:100AA00002EF05F0375E3EBC33AE15EF05F0D8809F
:100AB000800E33643430E86A342235223622D8A0DE
:100AC00015EF05F0363235323432374AF8EF04F09C
:100AD00015EF05F034C039F036C03BF0D89036340D
:100AE0009F0FF66E0C0EF76AF722000EF86AF822D6
:100AF0000A00F5503302F3CF33F0F4CF34F035026F
:100B0000F3CF35F0F4CF36F03902F3503426F450F9
:100B10003526F5503B02F35036260800F5504FEFCE
:100B200005F03550366EFF0BD8B4DAEF05F034C05F
:100B300035F033C034F0336A3650F00BD8B4BAEF26
:100B400005F0080E36BE4FEF05F0D8903436353636
:100B50003636E82A36BE4FEF05F0343635363636AF
:100B6000E82A36BE4FEF05F0343635363636E82AF9
:100B70004FEF05F035C03AF0D89036349F0FF66E3F
:100B80000C0EF76AF722000EF86AF8220A00F550F8
:100B90003402F3CF34F0F4CF35F03602F3CF36F031
:100BA0003A02F3503526F45036260800F550080F67
:100BB0004FEF05F03450366EFF0BD8B41AEF06F045
:100BC00033C035F0346A336A3650F00BD8B4FFEFD7
:100BD00005F0100E36BE4FEF05F0D890353636369C
:100BE000E82A36BE4FEF05F035363636E82A36BEEF
:100BF0004FEF05F035363636E82A4FEF05F036C0B0
:100C00003BF0D89036349F0FF66E0C0EF76AF72241
:100C1000000EF86AF8220A00F5503502F3CF35F0DD
:100C2000F4CF36F03B02F35036260800F550100F93
:100C30004FEF05F03350366EFF0BD8B40FEF05F0D1
:100C4000356A346A336A3650F00BD8B43BEF06F09D
:100C5000180E36BE4FEF05F0D8903636E82A36BE6D
:100C60004FEF05F03636E82A36BE4FEF05F0363640
:100C7000E82A4FEF05F0D89036349F0FF66E0C0E31
:100C8000F76AF722000EF86AF8220A00F5503602D9
:100C9000F3CF36F00800F550180F4FEF05F00000C5
:100CA0000780064006400520052005200520041089
:100CB00004100410041004100410041004103B7EEF
:100CC00036503B18426E336A37503C644FEF07F0A2
:100CD0003BC03DF03B8E368E37C041F03CC037F014
:100CE000E86A4164A1EF06F041503C5ED8B441EFA0
:100CF00007F0070E3C640FEF07F03C5E34C033F0A2
:100D000035C034F036C035F0366A3C4E41EF07F05E
:100D10003C64E4EF06F03C5E34C033F035C034F0A0
:100D2000356A3C4E41EF07F03C64C2EF06F03C5E92
:100D300034C033F0346A3C4E41EF07F03C64A9EF15
:100D400006F03DC036F03AC035F039C034F0336AB1
:100D5000000C030E3C64B4EF06F03C5E33380F0B1E
:100D6000336E3C4E41EF07F0D89033323C4E41EFAA
:100D700007F0D89033323C4E41EF07F0D890333231
:100D800041EF07F0030E3C64D3EF06F03C5E3338CE
:100D90000F0B336E3438F00B332634380F0B346EB0
:100DA0003C4E41EF07F0D890343233323C4E41EFA5
:100DB00007F0D890343233323C4E41EF07F0D890F0
:100DC0003432333241EF07F0030E3C64FBEF06F0A0
:100DD0003C5E33380F0B336E3438F00B3326343827
:100DE0000F0B346E3538F00B342635380F0B356E5B
:100DF0003C4E41EF07F0D8903532343233323C4E1E
:100E000041EF07F0D8903532343233323C4E41EF67
:100E100007F0D89035323432333241EF07F0030E09
:100E20003C642CEF07F03C5E33380F0B336E3438E4
:100E3000F00B332634380F0B346E3538F00B342674
:100E400035380F0B356E3638F00B352636380F0B2C
:100E5000366E3C4E41EF07F0D890363235323432A0
:100E600033323C4E41EF07F0D890363235323432CF
:100E700033323C4E41EF07F0D890363235323432BF
:100E80003332386A42AE30EF08F0336C341E351E10
:100E9000361EE86A34223522362230EF08F03C66EE
:100EA00053EF07F0000C386A36C03DF0368E3B8EAB
:100EB0003C50375C3C6ED8B424EF08F0070E3C641D
:100EC000F2EF07F03C5E39C038F03AC039F03BC071
:100ED0003AF03B6A3C4E24EF08F0070E3C64C7EF43
:100EE00007F03C5E39C038F03AC039F03A6A3C4EFF
:100EF00024EF08F0070E3C64A5EF07F03C5E39C014
:100F000038F0396A3C4E24EF08F0070E3C648CEF51
:100F100007F03DC036F0000C030E3C6497EF07F07D
:100F20003C5E38380F0B386E3C4E24EF08F0D890FA
:100F300038323C4E24EF08F0D89038323C4E24EF43
:100F400008F0D890383224EF08F0030E3C64B6EF76
:100F500007F03C5E38380F0B386E3938F00B382606
:100F600039380F0B396E3C4E24EF08F0D8903932E7
:100F700038323C4E24EF08F0D890393238323C4EAB
:100F800024EF08F0D8903932383224EF08F0030EFD
:100F90003C64DEEF07F03C5E38380F0B386E3938B2
:100FA000F00B382639380F0B396E3A38F00B3926EA
:100FB0003A380F0B3A6E3C4E24EF08F0D8903A3294
:100FC000393238323C4E24EF08F0D8903A32393278
:100FD00038323C4E24EF08F0D8903A323932383269
:100FE00024EF08F0030E3C640FEF08F03C5E383845
:100FF0000F0B386E3938F00B382639380F0B396E35
:101000003A38F00B39263A380F0B3A6E3B38F00B72
:101010003A263B380F0B3B6E3C4E24EF08F0D8903D
:101020003B323A32393238323C4E24EF08F0D89015
:101030003B323A32393238323C4E24EF08F0D89005
:101040003B323A3239323832336A42AE30EF08F04E
:10105000386C391E3A1E3B1EE86A39223A223B227E
:1010600038503326395034223A5035223B503622FC
:1010700042BE47EF08F0D8A053EF05F036323532C4
:1010800034323332373E53EF05F0F8EF04F0D8B086
:101090002CEF05F0E86A336C341E351E361E342200
:1010A000352236223D7E2CEF05F03F6AE86A3C642B
:1010B0000DEF05F037640FEF05F036503B183D6E2D
:1010C000368E3B8E3A343B344236D890E836423640
:1010D000B80FF66E130EF76E4250010BF722F86A46
:1010E000000EF8220A00F5CF31F00A00F5CF42F0E9
:1010F0000800F5CF41F03150415C316ED890393461
:101100003102F4CFF7FF3A343102F3CFE8FFF7268C
:10111000D8B0F42A406AF750405EF450415AE86A69
:10112000425A36C031F035C0F7FF34C0F6FF3450B4
:101130004002F4CF32F035504102F4CF34F0F3CF17
:1011400033F04002F3503226F4503322E86A34225E
:10115000F6504102F3503226F4503322E86A34222A
:1011600036504002F3503326F450342236504102B8
:10117000356AE86A3522F3503426F4503522F650A9
:101180004202F3503326F4503422366AE86A35229C
:101190003622F7504202F3503426F4503522E86AE2
:1011A000362231504202F3503526F450362236BEF4
:1011B000DFEF08F033363436353636363F063BC07F
:1011C00031F03AC0F7FF39C0F6FF39504002F4CF92
:1011D00032F03A504102F4CF39F0F3CF38F0400208
:1011E000F3503226F4503822E86A3922F650410290
:1011F000F3503226F4503822E86A39223B5040023C
:10120000F3503826F45039223B5041023A6AE86ADA
:101210003A22F3503926F4503A22F6504202F35063
:101220003826F45039223B6AE86A3A223B22F750CA
:101230004202F3503926F4503A22E86A3B223150F8
:101240004202F3503A26F4503B223BAE3BBC2FEF18
:1012500009F03236383639363A363B363F2A386C62
:10126000391E3A1E3B1EE86A39223A223B2236C01A
:1012700042F035C041F034C040F033C0F6FF345086
:101280003902F4CF32F035503802F450322635505E
:101290003902336AE86A3322F3503226F45033229B
:1012A000F6503A02F4503226346AE86A3322342285
:1012B00040503A02F3503226F4503322E86A342286
:1012C00041503A02F3503326F4503422365039025A
:1012D000F3503326F450342236503A02356AE86A25
:1012E0003522F3503426F450352242503802F35060
:1012F0003226F4503322E86A3422352242503B022F
:10130000F4CF36F0F3503526E86A3622F6503B0229
:10131000F3503226F4503322E86A34223522362242
:1013200040503B02F3503326F4503422E86A352211
:10133000362241503B02F3503426F4503522E86AFD
:10134000362236BEB1EF09F033363436353636360E
:101350003F0636BEB1EF09F0333634363536363611
:101360003F063C50375E800ED8A0BEEF09F03F2408
:101370003726D8B0F8EF04F0C3EF09F03F24372642
:10138000D8A002EF05F03EBC33AED8EF09F0D8800C
:10139000800E33643430E86A342235223622D8A0F5
:1013A000D8EF09F0363235323432374AF8EF04F0EC
:1013B0003DAE369E000CFFFF01FF04FE09FD10FC50
:1013C00019FB23FA30F93EF84EF760F674F58AF40B
:1013D000A1F3BAF2D5F1F1F00FF02FEF50EE73ED6B
:1013E00098ECBEEBE5EA0FEA39E966E893E7C3E675
:1013F000F3E526E559E48EE3C5E2FCE136E170E071
:10140000ACDFE9DE28DE68DDA9DCEBDB2FDB74DA9C
:10141000BAD902D94AD894D7DFD62CD679D5C7D431
:1014200017D468D3BAD20DD261D1B7D00DD064CF62
:10143000BDCE17CE71CDCDCC29CC87CBE6CA46CA5E
:10144000A6C908C96AC8CEC733C798C6FEC566C54F
:10145000CEC437C4A1C30CC378C2E5C152C1C1C058
:1014600030C0A0BF11BF83BEF6BD69BDDDBC52BC9C
:10147000C8BB3FBBB6BA2FBAA8B921B99CB817B838
:1014800093B710B78DB60BB68AB50AB58AB40BB44C
:101490008DB30FB392B216B29BB120B1A6B02CB0EF
:1014A000B3AF3BAFC3AE4CAED6AD60ADEBAC77AC3B
:1014B00003AC8FAB1DABABAA39AAC8A958A9E8A841
:1014C00079A80BA89CA72FA7C2A656A6EAA57FA518
:1014D00014A5AAA440A4D7A36EA306A39FA238A2D2
:1014E000D1A16BA106A1A1A03CA0D89F749F119F80
:1014F000AF9E4D9EEB9D8A9D299DC99C699C0A9C2F
:10150000AB9B4C9BEE9A919A349AD7997B991F99F1
:10151000C49869980E98B4975A970197A8965096D0
:10152000F895A0954995F2949C944694F0939B93DA
:101530004693F1929D924992F691A3915091FE901B
:10154000AC905A900990B88F688F178FC88E788E9C
:10155000298EDA8D8C8D3E8DF08CA38C568C098C67
:10156000BC8B708B248BD98A8E8A438AF889AE898A
:1015700064891B89D28889884088F887AF87688703
:101580002087D98692864C860586BF8579853485E5
:10159000EF84AA8465842184DD8399835683128332
:1015A000CF828D824A820882C681858143810281F1
:1015B000C180818040800180336AE86A3C62376480
:1015C0000FEF05F036503B183D6E3C5037267E0E2F
:1015D000D8A0F1EF0AF0375ED8B0F8EF04F0F5EFDD
:1015E0000AF0375ED8A002EF05F0368E3B8E36C08B
:1015F00042F035C041F034C040F034503902F4CFED
:1016000032F035503A02F4CF34F0F3CF33F03902F0
:10161000F3503226F4503322E86A342240503A0222
:10162000F3503226F4503322E86A3422365039021D
:10163000F3503326F450342236503A02356AE86AC1
:101640003522F3503426F450352240503B02F350FB
:101650003326F4503422366AE86A35223622415065
:101660003B02F3503426F4503522E86A36224250C9
:101670003B02F3503526F450362236BE48EF0BF0CD
:1016800033363436353636363706D8B402EF05F001
:101690003EBC33AE5DEF0BF0D880800E3364343047
:1016A000E86A342235223622D8A05DEF0BF03632BC
:1016B00035323432374AF8EF04F03DAE369E000C36
:1016C00036C042F035C041F035503A02F4CF34F024
:1016D000F3CF33F036503B02F4CF36F0F3CF35F092
:1016E0003A02F3503426F4503522E86A362241504B
:1016F0003B02F3503426F4503522E86A36223BAEE2
:1017000086EF0BF04150355E4250365A42AE000C27
:101710003A50355E3B50365A000CE86A3764000C8C
:1017200036C03DF0368E8E0E375CE8AEE4EF04F046
:10173000E86C376E070E3764EDEF0BF0375E35C09F
:1017400034F036C035F0366A374E16EF0CF0070E1F
:101750003764CBEF0BF0375E35C034F0356A374E67
:1017600016EF0CF0030E3764BDEF0BF0375E343824
:101770000F0B346E374E16EF0CF0D8903432374ED4
:1017800016EF0CF0D8903432374E16EF0CF0D8909C
:10179000343216EF0CF0030E3764DCEF0BF0375EDB
:1017A00034380F0B346E3538F00B342635380F0BC8
:1017B000356E374E16EF0CF0D89035323432374E46
:1017C00016EF0CF0D89035323432374E16EF0CF05D
:1017D000D8903532343216EF0CF0030E376404EF34
:1017E0000CF0375E34380F0B346E3538F00B34267E
:1017F00035380F0B356E3638F00B352636380F0B73
:10180000366E374E16EF0CF0D89036323532343211
:10181000374E16EF0CF0D890363235323432374E20
:1018200016EF0CF0D8903632353234323EBC34AE3E
:1018300024EF0CF0D880800E34643530E86A35220D
:10184000362236BEE4EF04F03DAE000C356C361E99
:10185000E86A3622000C3B503618E8BE65EF0CF003
:101860003BBE4CEF0CF03C50375CD8A0000CD8A429
:10187000010C3B50365CD8A0000CD8A4010C3A50A7
:10188000355CD8A0000CD8A4010C3950345CD8A029
:10189000000CD8A4010C000C37503C5CD8A0000C04
:1018A000D8A4010C36503B5CD8A0000CD8A4010C85
:1018B00035503A5CD8A0000CD8A4010C3450395CE7
:1018C000D8A0000CD8A4010C000C36AE010C000C02
:1018D00036503B18E8BEA2EF0CF036BE89EF0CF094
:1018E00037503C5CD8A0000CD8A4010C36503B5CAF
:1018F000D8A0000CD8A4010C35503A5CD8A0000C3C
:10190000D8A4010C3450395CD8A0000CD8A4010C28
:10191000000C3C50375CD8A0000CD8A4010C3B5004
:10192000365CD8A0000CD8A4010C3A50355CD8A085
:10193000000CD8A4010C3950345CD8A0000CD8A4F9
:0A194000010C000C3BAE010C000C82
:06194A00D9CFE6FFE1CF5A
:10195000D9FF060EE126A390A0909D90A092040EC0
:10196000BBCFDBFF050EBCCFDBFF0701CF6BD06B1E
:10197000D16BD26B040EDBCF04F0050EDBCF05F08C
:10198000066A076ACDC708F0CEC709F00A6A0B6A73
:101990000850045C006E09500558016E0A50065844
:1019A000026E0B500758036E00C0DFFF010E01C02E
:1019B000DBFF020E02C0DBFF030E03C0DBFF040EE1
:1019C000DBCFCDF7050EDBCFCEF7046805680668E0
:1019D0000768D9CFE9FFDACFEAFFEE50045C006E6A
:1019E000EE500558016EEE500658026EEE50075844
:1019F000036E0050D35D0150D4590250D5590350A5
:101A0000D6590CE2DF50D327010EDB50D423020E4F
:101A1000DB50D523030EDB50D62304D0D369D46921
:101A2000D569D6698650010B006E8450800B01E0A9
:101A3000010E00181DE0C72B000EC823FD0E396EE5
:101A4000AD0E3A6E3B6A790E3C6ED7C734F0D8C7FC
:101A500035F0D9C736F0DAC737F060EC06F034C09D
:101A6000D7F735C0D8F736C0D9F737C0DAF71CD06A
:101A7000C707000EC85BFD0E396EAD0E3A6E3B6AAD
:101A8000790E3C6ED7C734F0D8C735F0D9C736F0D9
:101A9000DAC737F05FEC06F034C0D7F735C0D8F7B7
:101AA00036C0D9F737C0DAF7BA70A380A0809D801E
:101AB000A082A190D9CFE1FFE552E7CFD9FF120074
:101AC000D9CFE6FFE1CFD9FF060EE126A390A09083
:101AD0009D90A092040EB8CFDBFF050EB9CFDBFFBF
:101AE0000701CF6BD06BD16BD26B040EDBCF04F050
:101AF000050EDBCF05F0066A076ACDC708F0CEC732
:101B000009F00A6A0B6A0850045C006E0950055817
:101B1000016E0A500658026E0B500758036E00C043
:101B2000DFFF010E01C0DBFF020E02C0DBFF030E70
:101B300003C0DBFF040EDBCFCDF7050EDBCFCEF706
:101B40000468056806680768D9CFE9FFDACFEAFFBD
:101B5000EE50045C006EEE500558016EEE500658D3
:101B6000026EEE500758036E0050D35D0150D459F9
:101B70000250D5590350D6590CE2DF50D327010E3D
:101B8000DB50D423020EDB50D523030EDB50D623CB
:101B900004D0D369D469D569D6698650010B006E2B
:101BA0008450800B01E0010E00181DE0C707000EF5
:101BB000C85BFD0E396EAD0E3A6E3B6A790E3C6E17
:101BC000D7C734F0D8C735F0D9C736F0DAC737F001
:101BD0005FEC06F034C0D7F735C0D8F736C0D9F778
:101BE00037C0DAF71CD0C72B000EC823FD0E396EA4
:101BF000AD0E3A6E3B6A790E3C6ED7C734F0D8C74B
:101C000035F0D9C736F0DAC737F060EC06F034C0EB
:101C1000D7F735C0D8F736C0D9F737C0DAF7B7707D
:101C2000A380A0809D80A082A490D9CFE1FFE5523F
:101C3000E7CFD9FF1200D9CFE6FFE1CFD9FF060EDB
:101C4000E126A392A3949D90A092040E74CFDBFF93
:101C5000050E75CFDBFF0701E36BE46BE56BE66B0D
:101C6000040EDBCF04F0050EDBCF05F0066A076A31
:101C7000E1C708F0E2C709F00A6A0B6A0850045C81
:101C8000006E09500558016E0A500658026E0B503E
:101C90000758036E00C0DFFF010E01C0DBFF020E1C
:101CA00002C0DBFF030E03C0DBFF040EDBCFE1F756
:101CB000050EDBCFE2F70468056806680768D9CF30
:101CC000E9FFDACFEAFFEE50045C006EEE500558F3
:101CD000016EEE500658026EEE500758036E00502B
:101CE000E75D0150E8590250E9590350EA590CE206
:101CF000DF50E727010EDB50E823020EDB50E9231B
:101D0000030EDB50EA2304D0E769E869E969EA6970
:101D10008650100B01E0010E006E8650080B01E0AA
:101D2000010E00181DE0DB2B000EDC23FD0E396ECA
:101D3000AD0E3A6E3B6A790E3C6EEBC734F0ECC7E1
:101D400035F0EDC736F0EEC737F060EC06F034C082
:101D5000EBF735C0ECF736C0EDF737C0EEF71CD027
:101D6000DB07000EDC5BFD0E396EAD0E3A6E3B6A92
:101D7000790E3C6EEBC734F0ECC735F0EDC736F0AA
:101D8000EEC737F05FEC06F034C0EBF735C0ECF788
:101D900036C0EDF737C0EEF77370A382A3849D8041
:101DA000A082A492D9CFE1FFE552E7CFD9FF12007C
:101DB000D9CFE6FFE1CFD9FF060EE126A392A39487
:101DC0009D90A092040E71CFDBFF050E72CFDBFF5A
:101DD0000701E36BE46BE56BE66B040EDBCF04F00D
:101DE000050EDBCF05F0066A076AE1C708F0E2C717
:101DF00009F00A6A0B6A0850045C006E0950055825
:101E0000016E0A500658026E0B500758036E00C050
:101E1000DFFF010E01C0DBFF020E02C0DBFF030E7D
:101E200003C0DBFF040EDBCFE1F7050EDBCFE2F7EB
:101E30000468056806680768D9CFE9FFDACFEAFFCA
:101E4000EE50045C006EEE500558016EEE500658E0
:101E5000026EEE500758036E0050E75D0150E859DE
:101E60000250E9590350EA590CE2DF50E727010E0E
:101E7000DB50E823020EDB50E923030EDB50EA239C
:101E800004D0E769E869E969EA698650100B01E066
:101E9000010E006E8650080B01E0010E00181DE0D7
:101EA000DB07000EDC5BFD0E396EAD0E3A6E3B6A51
:101EB000790E3C6EEBC734F0ECC735F0EDC736F069
:101EC000EEC737F05FEC06F034C0EBF735C0ECF747
:101ED00036C0EDF737C0EEF71CD0DB2B000EDC234D
:101EE000FD0E396EAD0E3A6E3B6A790E3C6EEBC755
:101EF00034F0ECC735F0EDC736F0EEC737F060ECE4
:101F000006F034C0EBF735C0ECF736C0EDF737C05C
:101F1000EEF77070A382A3849D80A082A494D9CF91
:101F2000E1FFE552E7CFD9FF1200D9CFE6FFE1CFBD
:101F3000D9FF040EE126A392A394A390A0909D90B4
:101F400004680568066A076ACDC708F0CEC709F0BD
:101F50000A6A0B6A0850045C006E09500558016E4D
:101F60000A500658026E0B500758036E00C0DFFF80
:101F7000010E01C0DBFF020E02C0DBFF030E03C037
:101F8000DBFF0701CD6BCE6B046805680668076848
:101F9000D9CFE9FFDACFEAFFEE50045C006EEE50D5
:101FA0000558016EEE500658026EEE500758036E4B
:101FB0000050CF5D0150D0590250D1590350D25931
:101FC0000CE2DF50CF27010EDB50D023020EDB5096
:101FD000D123030EDB50D22304D0CF69D069D1695D
:101FE000D2690468056806680768D9CFE9FFDACFC7
:101FF000EAFFEE50045C006EEE500558016EEE50A4
:102000000658026EEE500758036E0050D35D015023
:10201000D4590250D5590350D6590CE2DF50D3277A
:10202000010EDB50D423020EDB50D523030EDB5010
:10203000D62304D0D369D469D569D6690468056804
:10204000066A076AE1C708F0E2C709F00A6A0B6A84
:102050000850045C006E09500558016E0A5006587D
:10206000026E0B500758036E00C0DFFF010E01C067
:10207000DBFF020E02C0DBFF030E03C0DBFFE16BE0
:10208000E26B0468056806680768D9CFE9FFDACF14
:10209000EAFFEE50045C006EEE500558016EEE5003
:1020A0000658026EEE500758036E0050E35D015073
:1020B000E4590250E5590350E6590CE2DF50E3279A
:1020C000010EDB50E423020EDB50E523030EDB5050
:1020D000E62304D0E369E469E569E6690468056814
:1020E00006680768D9CFE9FFDACFEAFFEE50045C53
:1020F000006EEE500558016EEE500658026EEE501E
:102100000758036E0050E75D0150E8590250E95945
:102110000350EA590CE2DF50E727010EDB50E823B9
:10212000020EDB50E923030EDB50EA2304D0E769FB
:10213000E869E969EA69A382A384A380A0809D80FD
:10214000A192D9CFE1FFE552E7CFD9FF1200BA96AD
:10215000BA84BA92BA80968EA080A290A190120002
:10216000B796B784B792B7809880A380A590A490C3
:10217000120073967384739273809886A382A592DB
:10218000A492120070967084709270809888A384D4
:10219000A594A4941200B16AB18AB188B18CB186B9
:1021A000B18EA292B192A082B1801200D9CFE6FF87
:1021B000E1CFD9FF040EE126A090A390A092000EDB
:1021C000D8800701D355000ED455000ED555000E0A
:1021D000D65501E3FED0C751C81101E087D0E80E03
:1021E000046E650E056E190E066E8D0E076EC9C75C
:1021F00035F0CAC736F071EC04F034C008F035C0D1
:1022000009F036C00AF037C00BF008C039F009C039
:102210003AF00AC03BF00BC03CF004C034F005C0FB
:1022200035F006C036F007C037F0DCEC0AF034C0F9
:1022300000F035C001F036C002F037C003F0D3C75C
:1022400033F0D4C734F0D5C735F0D6C736F018EC24
:1022500005F034C010F035C011F036C012F037C0B0
:1022600013F0B2CF35F0B3CF36F06AEC04F034C0DF
:1022700014F035C015F036C016F037C017F014C092
:1022800039F015C03AF016C03BF017C03CF010C052
:1022900034F011C035F012C036F013C037F060ECE6
:1022A00006F034C00CF035C00DF036C00EF037C06B
:1022B0000FF00CC039F00DC03AF00EC03BF00FC06B
:1022C0003CF000C034F001C035F002C036F003C06D
:1022D00037F055EC08F034C0DEFF35C0DEFF36C005
:1022E000DEFF37C0DDFFDD52DD5272D0E80E046E36
:1022F000650E056E190E066E8D0E076EC7C735F09A
:10230000C8C736F071EC04F034C008F035C009F0ED
:1023100036C00AF037C00BF008C039F009C03AF0F7
:102320000AC03BF00BC03CF004C034F005C035F0EF
:1023300006C036F007C037F0DCEC0AF034C000F01D
:1023400035C001F036C002F037C003F0D3C733F018
:10235000D4C734F0D5C735F0D6C736F018EC05F041
:1023600034C00CF035C00DF036C00EF037C00FF0A1
:102370000CC039F00DC03AF00EC03BF00FC03CF07D
:1023800000C034F001C035F002C036F003C037F0B1
:1023900055EC08F034C0DEFF35C0DEFF36C0DEFF8E
:1023A00037C0DDFFDD52DD52CFC7D3F7D0C7D4F73A
:1023B000D1C7D5F7D2C7D6F70701800EC81503E0FD
:1023C000C969CA6903D0010EC96FCA6BC76BC86BF4
:1023D00006D0DE6ADE6ADE6ADD6ADD52DD52A0808A
:1023E000A380A082DECF33F0DECF34F0DECF35F035
:1023F000DDCF36F0DD52DD5200D0D9CFE1FFE5521E
:10240000E7CFD9FF1200D9CFE6FFE1CFD9FF040E05
:10241000E126A392A394A092000ED8800701E7556D
:10242000000EE855000EE955000EEA5501E3FED016
:10243000DB51DC1101E087D0E80E046E650E056EFD
:10244000190E066E8D0E076EDDC735F0DEC736F04D
:1024500071EC04F034C008F035C009F036C00AF061
:1024600037C00BF008C039F009C03AF00AC03BF0A1
:102470000BC03CF004C034F005C035F006C036F0A7
:1024800007C037F0DCEC0AF034C000F035C001F0D2
:1024900036C002F037C003F0E7C733F0E8C734F0C6
:1024A000E9C735F0EAC736F018EC05F034C010F093
:1024B00035C011F036C012F037C013F0B2CF35F08E
:1024C000B3CF36F06AEC04F034C014F035C015F028
:1024D00036C016F037C017F014C039F015C03AF006
:1024E00016C03BF017C03CF010C034F011C035F0FE
:1024F00012C036F013C037F060EC06F034C00CF0B8
:1025000035C00DF036C00EF037C00FF00CC039F0FA
:102510000DC03AF00EC03BF00FC03CF000C034F0EC
:1025200001C035F002C036F003C037F055EC08F0BA
:1025300034C0DEFF35C0DEFF36C0DEFF37C0DDFF52
:10254000DD52DD5272D0E80E046E650E056E190E76
:10255000066E8D0E076EDBC735F0DCC736F071EC0A
:1025600004F034C008F035C009F036C00AF037C0B6
:102570000BF008C039F009C03AF00AC03BF00BC0BC
:102580003CF004C034F005C035F006C036F007C09A
:1025900037F0DCEC0AF034C000F035C001F036C092
:1025A00002F037C003F0E7C733F0E8C734F0E9C7FB
:1025B00035F0EAC736F018EC05F034C00CF035C041
:1025C0000DF036C00EF037C00FF00CC039F00DC062
:1025D0003AF00EC03BF00FC03CF000C034F001C038
:1025E00035F002C036F003C037F055EC08F034C0C7
:1025F000DEFF35C0DEFF36C0DEFF37C0DDFFDD5257
:10260000DD52E3C7E7F7E4C7E8F7E5C7E9F7E6C750
:10261000EAF70701800EDC1503E0DD69DE6903D00F
:10262000010EDD6FDE6BDB6BDC6B06D0DE6ADE6A13
:10263000DE6ADD6ADD52DD52A382A384A082DECF92
:1026400033F0DECF34F0DECF35F0DDCF36F0DD52C3
:10265000DD5200D0D9CFE1FFE552E7CFD9FF12001C
:10266000D9CFE6FFE1CFD9FFA398FE0EDB5042C3DE
:10267000E9FF43C3EAFFEF6E03014051421902E153
:102680004151431905E13EC342F33FC343F303D035
:10269000422B000E4323A388E552E7CFD9FF120057
:1026A000D9CFE6FFE1CFD9FFFD0EDBCFE9FFFE0E6C
:1026B000DBCFEAFFEF5010E0FD0EDBCFE9FFFE0EAF
:1026C000DBCFEAFFEF50E66ECBDFE552FD0EDB2AF3
:1026D000FE0E01E3DB2AE8D70D0EE66EC1DFE55200
:1026E0000A0EE66EBDDFE552E552E7CFD9FF1200D4
:1026F000D9CFE6FFE1CFD9FF020EE126DE6ADD6A1F
:10270000DECF00F0DDCF01F0FB0EDBCF02F0FC0EE0
:10271000DBCF03F001500318E8AE02D0033404D03D
:102720000250005C0350015814E2FD0EDBCFE9FFBC
:10273000FE0EDBCFEAFFEF50E66E92DFE552FD0EB4
:10274000DB2AFE0E01E3DB2ADF2A010E01E3DB2A8E
:10275000D7D7D9CFE1FFE552E7CFD9FF1200D9CFC4
:10276000E6FFE1CFD9FF040EE126FB0EDBCF00F040
:10277000FC0EDBCF01F0FD0EDBCF02F0FE0EDBCF57
:1027800003F0396A3A6A3B6A3C6A00C034F001C01F
:1027900035F002C036F003C037F068EC0CF0010AE7
:1027A0002DE1FB0EDBCF00F0FC0EDBCF01F0FD0EC8
:1027B000DBCF02F0FE0EDBCF03F0396A3A6A800EFF
:1027C0003B6E7F0E3C6E00C034F001C035F002C09D
:1027D00036F003C037F0DCEC0AF0FB0E34C0DBFF50
:1027E000FC0E35C0DBFFFD0E36C0DBFFFE0E37C032
:1027F000DBFF2D0EE66E34DFE55204D02B0EE66EC5
:102800002FDFE552FB0EDBCF34F0FC0EDBCF35F0D3
:10281000FD0EDBCF36F0FE0EDBCF37F08DEC0BF08C
:1028200035C0DEFF36C0DDFFDECF00F0DDCF01F0CA
:102830000050E66E15DFE552DECF00F0DDCF01F08F
:1028400001C000F0016A0050E66E0ADFE5522E0E6C
:10285000E66E06DFE552FB0EDBCF04F0FC0EDBCFAD
:1028600005F0FD0EDBCF06F0FE0EDBCF07F0000E0D
:10287000DFCF35F0010EDBCF36F071EC04F034C061
:1028800008F035C009F036C00AF037C00BF008C0B8
:1028900039F009C03AF00AC03BF00BC03CF004C06C
:1028A00034F005C035F006C036F007C037F05FECF5
:1028B00006F034C000F035C001F036C002F037C079
:1028C00003F0396A3A6A3B6A8F0E3C6E00C034F0FE
:1028D00001C035F002C036F003C037F0DCEC0AF07E
:1028E000FB0E34C0DBFFFC0E35C0DBFFFD0E36C037
:1028F000DBFFFE0E37C0DBFFFB0EDBCF34F0FC0E40
:10290000DBCF35F0FD0EDBCF36F0FE0EDBCF37F040
:102910008DEC0BF0020E35C0DBFF030E36C0DBFF83
:10292000FF0EE76E020EDBCF00F0030EDBCF01F0EF
:10293000E7500016016A0050E66E92DEE552020E84
:10294000DBCF00F0030EDBCF01F001C000F0016A25
:102950000050E66E85DEE552D9CFE1FFE552E7CFC4
:10296000D9FF1200D9CFE6FFE1CFD9FF0A0EE12649
:102970002D0EF36E040EF3CFDBFF2D0EF36E050E5E
:10298000F3CFDBFF2D0EF36E060EF3CFDBFF2D0E24
:10299000F36E070EF3CFDBFF2D0EF36E080EF3CFB1
:1029A000DBFF090EDB6AFB0EDBCF00F0FC0EDBCF9A
:1029B00001F0FD0EDBCF02F0FE0EDBCF03F0396A33
:1029C0003A6A3B6A3C6A00C034F001C035F002C08C
:1029D00036F003C037F068EC0CF0010A2CE1FB0E76
:1029E000DBCF00F0FC0EDBCF01F0FD0EDBCF02F001
:1029F000FE0EDBCF03F0396A3A6A800E3B6E7F0E23
:102A00003C6E00C034F001C035F002C036F003C0A7
:102A100037F0DCEC0AF0FB0E34C0DBFFFC0E35C0F7
:102A2000DBFFFD0E36C0DBFFFE0E37C0DBFF2D0ED9
:102A3000E66E16DEE552FB0EDBCF34F0FC0EDBCF8C
:102A400035F0FD0EDBCF36F0FE0EDBCF37F08DEC30
:102A50000BF035C0DEFF36C0DDFFDECF00F0DDCF8E
:102A600001F00150030AE8AE02D0013405D0E80EAF
:102A7000D8800054030E015409E2D950040FE66EC9
:102A8000DACFE6FF0DDEE552E55218D1D950040F3A
:102A9000E66EDACFE6FFDECFE6FFDDCFE6FFCDEC78
:102AA00022F0E552E552E552E552020EDB6A030ED2
:102AB000DB6AD950040F006EDACF01F0020EDB5052
:102AC0000024E96E030EDB500120EA6EEF5017E0A0
:102AD000D950040F006EDACF01F0020EDB50002453
:102AE000E96E030EDB500120EA6EEF50E66EB8DDB2
:102AF000E552020EDB2A030E01E3DB2ADAD72E0EA3
:102B0000E66EAEDDE552FB0EDBCF00F0FC0EDBCF58
:102B100001F0FD0EDBCF02F0FE0EDBCF03F0000E66
:102B2000DFCF35F0010EDBCF36F071EC04F034C0AE
:102B300004F035C005F036C006F037C007F004C019
:102B400039F005C03AF006C03BF007C03CF000C0C9
:102B500034F001C035F002C036F003C037F05FEC4E
:102B600006F0FB0E34C0DBFFFC0E35C0DBFFFD0EB4
:102B700036C0DBFFFE0E37C0DBFF020EDB6A030E42
:102B8000DB6A020EDBCF00F0030EDBCF01F0015059
:102B9000000AE8AE02D0D89004D0030E005C000E0C
:102BA000015801E383D0FB0EDBCF00F0FC0EDBCF3E
:102BB00001F0FD0EDBCF02F0FE0EDBCF03F0396A31
:102BC0003A6A200E3B6E820E3C6E00C034F001C0AB
:102BD00035F002C036F003C037F0DCEC0AF0FB0E33
:102BE00034C0DBFFFC0E35C0DBFFFD0E36C0DBFF63
:102BF000FE0E37C0DBFFFB0EDBCF34F0FC0EDBCF6D
:102C000035F0FD0EDBCF36F0FE0EDBCF37F08DEC6E
:102C10000BF035C0DEFF36C0DDFFDECF00F0DDCFCC
:102C200001F0300E0024E66E1BDDE552FB0EDBCF1B
:102C300000F0FC0EDBCF01F0FD0EDBCF02F0FE0E4C
:102C4000DBCF03F0000EDFCF35F0010EDBCF36F027
:102C500071EC04F034C004F035C005F036C006F065
:102C600037C007F004C039F005C03AF006C03BF0A9
:102C700007C03CF000C034F001C035F002C036F0AF
:102C800003C037F05FEC06F0FB0E34C0DBFFFC0E38
:102C900035C0DBFFFD0E36C0DBFFFE0E37C0DBFFAD
:102CA000020EDB2A030E01E3DB2A6BD70D0EE66E64
:102CB000D7DCE5520A0EE66ED3DCE552D9CFE1FF50
:102CC000E552E7CFD9FF1200D9CFE6FFE1CFD9FF18
:102CD000020EE126A39A6BA20BD06B986B88FD0EB7
:102CE000DBCFE9FFFE0EDBCFEAFFEF6ADE68DD68CF
:102CF00003013A513C1902E13B513D190AE1FD0E35
:102D0000DBCFE9FFFE0EDBCFEAFFEF6ADE6ADD6AAA
:102D100020D03AC3E9FF3BC3EAFFEF50E66EFD0E59
:102D2000DBCFE9FFFE0EDBCFEAFFE552E750EF6EA7
:102D300038513A1902E139513B1905E136C33AF3EA
:102D400037C33BF303D03A2B000E3B23010EDE6E5C
:102D5000DD6AA38ADECF00F0DDCF01F000C0F3FF13
:102D600001C0F4FF00D0D9CFE1FFE552E7CFD9FF92
:102D700012006E503CC3E9FF3DC3EAFFEF6E6BB437
:102D80000FD0030138513C1902E139513D1905E1D9
:102D900036C33CF337C33DF303D03C2B000E3D2339
:102DA000A49A120003014451421902E1455143190A
:102DB00002E1A39814D044C3E9FF45C3EAFFEF50F2
:102DC0006D6E4051441902E14151451905E13EC380
:102DD00044F33FC345F303D0442B000E45231200B8
:102DE000D9CFE6FFE1CFD9FFE6520301000E3E6FD7
:102DF000020E3F6FFF0E406F020E416F3EC342F363
:102E00003FC343F33EC344F33FC345F3000E366F65
:102E1000010E376FFF0E386F010E396F36C33AF36C
:102E200037C33BF336C33CF337C33DF3150EE66EB1
:102E3000FC0EE66EE3EC23F0E552E552A598A59A68
:102E4000989298846E50DF6E6E50DF6EA49AE552B1
:082E5000E552E7CFD9FF1200A3
:082E5800DACFE4FFE2CFDAFF5C
:102E6000E9CFE4FFEACFE4FFE652F2A202D09CD819
:102E700002D09EB6C8D8E552E5CFEAFFE5CFE9FF1C
:102E8000E5CFDAFF1100E66A010EE66E050EE66E8A
:102E9000B6EC23F0E552E552E5521200070EB46E8F
:102EA000000E886E876E866E856E846E836E826E6F
:102EB000816E806E916E906E8F6E8E6E8D6E8C6E4A
:102EC0008B6E8A6E896E92689368BF0E946E956A57
:102ED000700E966E9F0E976EE40E986E0F0E996EA2
:102EE0009A68C16E070EC06EF19EB0989C8EA26A61
:102EF0009F6AA06A9D6AA36AA56AC5DF9F86D08E75
:102F00009E969D869382F06AF288F09EF098F192E8
:102F1000F09AF16AF28CF28E1200D9CFE6FFE1CF7F
:102F2000D9FFE652BBDF07019897989903015C0E21
:102F3000516F070E526FDF6A100EDF5C0AE2DF503E
:102F4000EA6A5125E96E5251EA227F0EEF6EDF2ABE
:102F5000F3D70701756B010E766FC90E776F070106
:102F60009885010ED56E800ED76EF90ED66ED59E61
:102F7000580EE66E070EE66E94D8E552E55207014C
:102F80009893580EE66E070EE66E8BD8E552E55222
:102F900007019893E552E552E7CFD9FF12008282EC
:102FA0008088949292981200F2920301200E4D6F45
:102FB0009F86070198A906D00301E00E4A6F000E14
:102FC0004B6F05D00301C00E4A6F000E4B6F070117
:102FD00098A1987998A706D00301800E486F000E3B
:102FE000496F05D00301A00E486F000E496FC9CF8D
:102FF0004EF348C3E9FF49C3EAFF482B000E4923BB
:10300000EF50C96E12009E96C9CF4EF303014D5189
:10301000000823E24AC3E9FF4BC3EAFF4A2B000E34
:103020004B234EC3EFFF48C3E9FF49C3EAFF482BD8
:103030004923EFCF4EF34EC3C9FF4D074D510CE16D
:103040000701020E766F070198939881770ED76E6D
:10305000470ED66EF294D58E01D0C96A1200D9CF30
:10306000E6FFE1CFD9FF070198A117D0FD0EDBCF16
:10307000E6FFFE0EDBCFE6FF66EC20F0E552E55200
:103080009D96070198919D860F0E00012E5D05E02B
:103090006EC7E6FFB0EC1FF0E552E552E7CFD9FF6F
:1030A0001200D9CFE6FFE1CFD9FF070198B332D0A4
:1030B000FD0EDBCFE9FFFE0EDBCFEAFF1E0EE92699
:1030C000000EEA22EF50020809E1FD0EDBCFE6FF19
:1030D000FE0EDBCFE6FF69D8E552E552FD0EDBCFF1
:1030E000E9FFFE0EDBCFEAFF150EE926000EEA220D
:1030F000EF9EFD0EDBCFE6FFFE0EDBCFE6FFD4EC4E
:103100001FF0E552E5529D960701987798839D86BA
:103110000701752BE552E7CFD9FF12009D960701F5
:1031200098919D861200D9CFE6FFE1CFD9FF00012B
:103130002E6BD950FD0FE96EFF0EDA20EA6E010EFC
:10314000EE1801E1ED5002E12E8101D0BA6AD950AA
:10315000FB0FE96EFF0EDA20EA6E010EEE1801E1B8
:10316000ED5002E12E8301D0B76AD950F90FE96E14
:10317000FF0EDA20EA6E010EEE1801E1ED5002E1D9
:103180002E8501D0736AD950F70FE96EFF0EDA2051
:10319000EA6E010EEE1801E1ED5002E12E8701D03A
:1031A000706AE552E7CFD9FF1200D9CFE6FFE1CF31
:1031B000D9FFFD0EDBCFE9FFFE0EDBCFEAFF1C0ED1
:1031C000E926000EEA22EF6AFD0EDBCFE9FFFE0ED4
:1031D000DBCFEAFF170EE926000EEA22EF6AC6AE41
:1031E0000ED0C69EFD0EDBCFE9FFFE0EDBCFEAFF61
:1031F000170EE926000EEA22010EEF6E22D0F150E2
:10320000800B10E0F250080B0DE0FD0EDBCFE9FF64
:10321000FE0EDBCFEAFF170EE926000EEA22020EB1
:10322000EF6E0FD0F0A60DD0909EFD0EDBCFE9FF24
:10323000FE0EDBCFEAFF170EE926000EEA22030E90
:10324000EF6E250EC614250819E0FD0EDBCFE9FF51
:10325000FE0EDBCFEAFF1C0EE926000EEA22010E6D
:10326000EF6EFD0EDBCFE9FFFE0EDBCFEAFF170EA0
:10327000E926000EEA22C6CFEFFF80D1C55019E043
:10328000FD0EDBCFE9FFFE0EDBCFEAFF1C0EE926C9
:10329000000EEA22020EEF6EFD0EDBCFE9FFFE0EFE
:1032A000DBCFEAFF170EE926000EEA22C5CFEFFFBB
:1032B00065D1D0BE19D0FD0EDBCFE9FFFE0EDBCF0E
:1032C000EAFF1C0EE926000EEA22030EEF6EFD0E49
:1032D000DBCFE9FFFE0EDBCFEAFF170EE926000E7B
:1032E000EA22D0CFEFFF4AD19DB619D0FD0EDBCF39
:1032F000E9FFFE0EDBCFEAFF1C0EE926000EEA22F4
:10330000040EEF6EFD0EDBCFE9FFFE0EDBCFEAFF12
:10331000170EE926000EEA229DCFEFFF2FD19C5019
:1033200019E0FD0EDBCFE9FFFE0EDBCFEAFF1C0E3E
:10333000E926000EEA22050EEF6EFD0EDBCFE9FF57
:10334000FE0EDBCFEAFF170EE926000EEA229CCF25
:10335000EFFF14D1080E9F5C19E0FD0EDBCFE9FFF3
:10336000FE0EDBCFEAFF1C0EE926000EEA22060E57
:10337000EF6EFD0EDBCFE9FFFE0EDBCFEAFF170E8F
:10338000E926000EEA229FCFEFFFF8D0A25019E005
:10339000FD0EDBCFE9FFFE0EDBCFEAFF1C0EE926B8
:1033A000000EEA22070EEF6EFD0EDBCFE9FFFE0EE8
:1033B000DBCFEAFF170EE926000EEA22A2CFEFFFCD
:1033C000DDD0A55019E0FD0EDBCFE9FFFE0EDBCF0F
:1033D000EAFF1C0EE926000EEA22080EEF6EFD0E33
:1033E000DBCFE9FFFE0EDBCFEAFF170EE926000E6A
:1033F000EA22A5CFEFFFC2D0100EF214100819E098
:10340000FD0EDBCFE9FFFE0EDBCFEAFF1C0EE92647
:10341000000EEA22090EEF6EFD0EDBCFE9FFFE0E75
:10342000DBCFEAFF170EE926000EEA22F2CFEFFF0C
:10343000A5D0470EF11419E0FD0EDBCFE9FFFE0E1B
:10344000DBCFEAFF1C0EE926000EEA220A0EEF6E21
:10345000FD0EDBCFE9FFFE0EDBCFEAFF170EE926FC
:10346000000EEA22F1CFEFFF89D0C00EF01419E070
:10347000FD0EDBCFE9FFFE0EDBCFEAFF1C0EE926D7
:10348000000EEA220B0EEF6EFD0EDBCFE9FFFE0E03
:10349000DBCFEAFF170EE926000EEA22F0CFEFFF9E
:1034A0006DD092A819D0FD0EDBCFE9FFFE0EDBCF69
:1034B000EAFF1C0EE926000EEA220C0EEF6EFD0E4E
:1034C000DBCFE9FFFE0EDBCFEAFF170EE926000E89
:1034D000EA2292CFEFFF52D093B019D0FD0EDBCF8E
:1034E000E9FFFE0EDBCFEAFF1C0EE926000EEA2202
:1034F0000D0EEF6EFD0EDBCFE9FFFE0EDBCFEAFF18
:10350000170EE926000EEA2293CFEFFF37D03E0ECA
:1035100094141C0819E0FD0EDBCFE9FFFE0EDBCF93
:10352000EAFF1C0EE926000EEA220E0EEF6EFD0EDB
:10353000DBCFE9FFFE0EDBCFEAFF170EE926000E18
:10354000EA2294CFEFFF1AD097BE18D0FD0EDBCF42
:10355000E9FFFE0EDBCFEAFF1C0EE926000EEA2291
:103560000F0EEF6EFD0EDBCFE9FFFE0EDBCFEAFFA5
:10357000170EE926000EEA2297CFEFFFE552E7CFBC
:04358000D9FF12005D
:0C358400D9CFE6FFE1CFD9FF040EE1260D
:10359000D950FB0FE96EFF0EDA20EA6EEECFE6FFA0
:1035A000EECFE6FFEECFE6FFEFCFE6FF7FD9E552A5
:1035B000E552E552E5521DD8DAD80FD933C0DEFF07
:1035C00034C0DEFF35C0DEFF36C0DDFFDD52DD5228
:1035D000DECF33F0DECF34F0DECF35F0DDCF36F0A6
:1035E000DD52DD5200D0D9CFE1FFE552E7CFD9FF60
:1035F0001200D9CFE6FFE1CFD9FF040EE126DE6A43
:10360000DD6ADECF00F0DDCF01F00150000AE8AE48
:1036100002D0D89004D0030E005C000E015801E3E4
:1036200090D0020EDB6A030EDB6A020EDBCF00F0E5
:10363000030EDBCF01F00150000AE8AE02D0D890B3
:1036400004D0030E005C000E015876E230C302F095
:1036500031C303F0060E0302F3CF03F00202F3CFEF
:1036600002F0F4500326000E0226030E0322020E7F
:10367000356E366ADBCF3AF0030EDBCF3BF060EC01
:103680000BF002503324E96E03503420EA6EEECF83
:1036900000F0EFCF01F0DF50001803E1DE52DD5003
:1036A000011844E1020EDBCFE9FF030EDBCFEAFF96
:1036B000D890E936EA36240EE926030EEA22010EF6
:1036C000EE1801E1ED5032E130C300F031C301F0FA
:1036D000060E0102F3CF01F00002F3CF00F0F45028
:1036E0000126120E0026030E0122020E356E366AE6
:1036F000DBCF3AF0030EDBCF3BF060EC0BF0005079
:103700003324E96E01503420EA6EEE50EFCFEAFF29
:10371000E96E010ED890E936EA36E806FBE12A0E9A
:10372000E926030EEA22010EEE6EED6A020EDB2A96
:10373000030E01E3DB2A79D7DF2A010E01E3DB2A3E
:1037400060D730C3E9FF31C3EAFF010ED890E936F4
:10375000EA36E806FBE12A0EE926030EEA22EE6AC3
:10376000ED6AD9CFE1FFE552E7CFD9FF1200D9CFFB
:10377000E6FFE1CFD9FF020EE126DE6ADD6ADECF89
:1037800000F0DDCF01F00150000AE8AE02D0D89081
:1037900004D0030E005C000E015819E2DECFE9FFF1
:1037A000DDCFEAFFD890E936EA362A0EE926030E85
:1037B000EA22010EEE1801E1ED5004E1DECF30F314
:1037C000DDCF31F3DF2A010E01E3DB2AD8D7D9CFD1
:1037D000E1FFE552E7CFD9FF1200D9CFE6FFE1CFF5
:1037E000D9FF040EE12630C3E9FF31C3EAFF010E21
:1037F000D890E936EA36E806FBE12A0EE926030E00
:10380000EA22010EEE1801E1ED5005E10301326BF1
:10381000336B346B356B020E0301301901E131510A
:1038200028E0010E301901E1315117E0305101E17A
:10383000315107E0DE6ADE6ADE6ADD6ADD52DD52A2
:1038400024D0CFD833C0DEFF34C0DEFF35C0DEFF6A
:1038500036C0DDFFDD52DD5218D0EFD833C0DEFFB9
:1038600034C0DEFF35C0DEFF36C0DDFFDD52DD5285
:103870000CD0CCD833C0DEFF34C0DEFF35C0DEFF55
:1038800036C0DDFFDD52DD5200D0DECF33F0DECFBB
:1038900034F0DECF35F0DDCF36F0DD52DD5200D032
:1038A000D9CFE1FFE552E7CFD9FF1200D9CFE6FF2C
:1038B000E1CFD9FF0301246B256BFB0EDBCF00F0BA
:1038C000FC0EDBCF01F0FD0EDBCF02F0FE0EDBCFF6
:1038D00003F0CD0E396ECC0E3A6E4C0E3B6E7A0E66
:1038E0003C6E00C034F001C035F002C036F003C0B9
:1038F00037F02BEC0CF0010A23E0FB0EDBCF04F0D9
:10390000FC0EDBCF05F0FD0EDBCF06F0FE0EDBCFAD
:1039100007F0CD0E396ECC0E3A6E3B6E7A0E3C6ED1
:1039200004C034F005C035F006C036F007C037F0EB
:1039300068EC0CF0010A04E0010E0301246F256B12
:103940000301266B276BFB0EDBCF00F0FC0EDBCFF9
:1039500001F0FD0EDBCF02F0FE0EDBCF03F0CD0E4B
:10396000396ECC0E3A6E3B6E7A0E3C6E00C034F06F
:1039700001C035F002C036F003C037F068EC0CF03F
:10398000010A04E1010E0301266F276B0301286B76
:10399000296BFB0EDBCF00F0FC0EDBCF01F0FD0E40
:1039A000DBCF02F0FE0EDBCF03F0CD0E396ECC0E76
:1039B0003A6E4C0E3B6E7A0E3C6E00C034F001C085
:1039C00035F002C036F003C037F02BEC0CF0010AE2
:1039D00004E1010E0301286F296BE552E7CFD9FFFF
:1039E0001200D9CFE6FFE1CFD9FF006A016A026A6F
:1039F000036A00C033F001C034F002C035F003C0E8
:103A000036F000D0E552E7CFD9FF1200D9CFE6FF5C
:103A1000E1CFD9FF006A016A800E026E7F0E036E4D
:103A200000C033F001C034F002C035F003C036F0FE
:103A300000D0E552E7CFD9FF1200D9CFE6FFE1CFA2
:103A4000D9FF006A016A026A7F0E036E00C033F07C
:103A500001C034F002C035F003C036F000D0E552AA
:063A6000E7CFD9FF1200C0
:0A3A6600D8CFE4FFE0CFE4FFE46EE8
:103A7000DACFE4FFE2CFDAFFE9CFE4FFEACFE4FFF9
:103A8000F3CFE4FFF4CFE4FFE652D9CFE6FFE1CF76
:103A9000D9FFE6529E50010B05E09D50010B02E05C
:103AA00027D811D0A450200B06E0A350200B03E030
:103AB000B9EC16F008D0A450100B05E0A350100B81
:103AC00002E0D2EC16F0E552E552E7CFD9FFE5521D
:103AD000E5CFF4FFE5CFF3FFE5CFEAFFE5CFE9FF60
:103AE000E5CFDAFFE550E5CFE0FFE5CFD8FF1000E6
:103AF000D9CFE6FFE1CFD9FF020EE126A50ECF6EAA
:103B0000320ECE6E8E70BCD8F3CFDEFFF4CFDDFF69
:103B1000D9CFE9FFDACFEAFF010EEE1801E1ED504F
:103B200002E10701C183396A3A6A200E3B6E810EB9
:103B30003C6EC2C734F0C3C735F0C4C736F0C5C742
:103B400037F02BEC0CF0010A36E10701C26BC36BB6
:103B5000C46BC56BC1A318D00B0EE66EE66AAD0E42
:103B6000E66E070EE66E78EC13F0E552E552E5528C
:103B7000E5520D0EE66E30EC13F0E5520A0EE66EDD
:103B800030EC13F0E55217D00D0EE66EE66A990E92
:103B9000E66E070EE66E78EC13F0E552E552E5525C
:103BA000E5520D0EE66E30EC13F0E5520A0EE66EAD
:103BB00030EC13F0E552A30E396E560E3A6E180E25
:103BC0003B6E790E3C6EC2C734F0C3C735F0C4C734
:103BD00036F0C5C737F060EC06F034C0C2F735C028
:103BE000C3F736C0C4F737C0C5F79E90D9CFE1FF01
:103BF000E552E7CFD9FF1200CD6ACD8ACD88A50E58
:103C0000CF6E320ECE6ECD8E9F909D80F2A4FED7E9
:103C1000F2B4FED7CD801200F28C1200F29C580E46
:103C2000E66E070EE66E51EC18F0E552E552CFEC69
:103C300017F0070198A1FDD7780EE66E070EE66E25
:103C40002FEC18F0E552E552D7DFF0EC16F0E4DF88
:103C5000990EE66E070EE66E50EC13F0E552E55253
:103C6000050EE66E30EC13F0E5522E0EE66E30ECEB
:103C700013F0E552020EE66E30EC13F0E55212003E
:103C8000D9CFE6FFE1CFD9FF030EE126010EDB6AB3
:103C9000020EDB6A010EDBCF00F0020EDBCF01F07B
:103CA0000150000AE8AE02D0D89004D0080E005CA3
:103CB000000E015801E301D1D9CFE6FFDACFE6FFCC
:103CC00064EC16F0E552E552F3CF00F0F4CF01F0CA
:103CD000010E001801E1015007E0006A016A00C00E
:103CE000F3FF01C0F4FFF0D00701C651140A01E14F
:103CF000D1D0070A01E1C6D0010A01E1BBD0030A15
:103D000001E1B0D0010A01E1A5D01F0A01E19AD07A
:103D1000010A01E18FD0030A01E184D0010A01E127
:103D200079D0070A6FE0010A65E0030A5BE0010A47
:103D300051E00F0A47E0010A3DE0030A33E0010ABF
:103D400029E0070A1FE0010A15E0030A0BE0010A57
:103D500001E0ADD0470EDF5C03E1010EC66F01D07C
:103D6000C66BA5D06F0EDF5C03E1020EC66F01D0FB
:103D7000C66B9DD06F0EDF5C03E1030EC66F01D0F2
:103D8000C66B95D0640EDF5C03E1040EC66F01D0F4
:103D9000C66B8DD0620EDF5C03E1050EC66F01D0ED
:103DA000C66B85D0790EDF5C03E1060EC66F01D0CD
:103DB000C66B7DD0650EDF5C03E1070EC66F01D0D8
:103DC000C66B75D02C0EDF5C03E1080EC66F01D008
:103DD000C66B6DD0200EDF5C03E1090EC66F01D00B
:103DE000C66B65D0430EDF5C03E10A0EC66F01D0DF
:103DF000C66B5DD0720EDF5C03E10B0EC66F01D0A7
:103E0000C66B55D0750EDF5C03E10C0EC66F01D09A
:103E1000C66B4DD0650EDF5C03E10D0EC66F01D0A1
:103E2000C66B45D06C0EDF5C03E10E0EC66F01D091
:103E3000C66B3DD0200EDF5C03E10F0EC66F01D0D4
:103E4000C66B35D0570EDF5C03E1100EC66F01D094
:103E5000C66B2DD06F0EDF5C03E1110EC66F01D073
:103E6000C66B25D0720EDF5C03E1120EC66F01D067
:103E7000C66B1DD06C0EDF5C03E1130EC66F01D064
:103E8000C66B15D0640EDF5C03E1140EC66F01D063
:103E9000C66B0DD0C66B2E0EDF5C08E1010E006E06
:103EA000016A00C0F3FF01C0F4FF0ED000D0010E84
:103EB000DB2A020E01E3DB2AEDD6006A016A00C0AC
:103EC000F3FF01C0F4FF00D0D9CFE1FFE552E7CF07
:103ED000D9FF1200070198A110D0780EE66E070EE8
:103EE000E66E2FEC18F0E552E552580EE66E070E1E
:103EF000E66E51EC18F0E552E55212008DEC17F029
:103F0000070198918BDE07016C83E4DFFED7120076
:103F1000000EE96EEA6E040095EC1FF0EA2A080E26
:103F2000EA5CD8A48BEF1FF01200EF6AE93E95EF30
:103F30001FF01200FF0EE3CF21F021380F0B060F08
:103F4000D8B2070F2A0FAD6E86EC21F021500F0B6F
:103F5000060FD8B2070F2A0FAD6E86EC21F0000CC9
:103F6000FF0EE3CF2DF02DB0968E2DA0969E2DB294
:103F700098802DA298902DB498862DA498962DB651
:103F800098882DA698982DB896802DA896902DBA31
:103F900096822DAA96922DBC96842DAC96942DBE19
:103FA00096862DAE96961200EACF1CF0E9CF1DF052
:103FB000FF0EE3CFEAFFFE0EE3CFE9FF98A741D063
:103FC000EECFA0F0EECFA1F0EECFA2F0EECFA3F0B7
:103FD000EECFA4F0EECFA5F0EECFA6F0EECFA7F097
:103FE000EECFA8F0EECFA9F0EECFAAF0EECFABF077
:103FF000EECFACF0EECFADF0EECFAEF0EECFAFF057
:10400000EECFB0F0EECFB1F0EECFB2F0EECFB3F036
:10401000EECFB4F0EECFB5F0EECFB6F0EECFB7F016
:10402000EECFB8F0EECFB9F0EECFBAF0EECFBBF0F6
:10403000EECFBCF0EECFBDF0EECFBEF0EECFBFF0D6
:1040400040D0EECF80F0EECF81F0EECF82F0EECF19
:1040500083F0EECF84F0EECF85F0EECF86F0EECF9A
:1040600087F0EECF88F0EECF89F0EECF8AF0EECF7A
:104070008BF0EECF8CF0EECF8DF0EECF8EF0EECF5A
:104080008FF0EECF90F0EECF91F0EECF92F0EECF3A
:1040900093F0EECF94F0EECF95F0EECF96F0EECF1A
:1040A00097F0EECF98F0EECF99F0EECF9AF0EECFFA
:1040B0009BF0EECF9CF0EECF9DF0EECF9EF0EECFDA
:1040C0009FF01CC0EAFF1DC0E9FF120098A112007A
:1040D000EACF1CF0E9CF1DF0FF0EE3CFEAFFFE0EA2
:1040E000E3CFE9FF98A941D0C0C0EEFFC1C0EEFF09
:1040F000C2C0EEFFC3C0EEFFC4C0EEFFC5C0EEFFFE
:10410000C6C0EEFFC7C0EEFFC8C0EEFFC9C0EEFFDD
:10411000CAC0EEFFCBC0EEFFCCC0EEFFCDC0EEFFBD
:10412000CEC0EEFFCFC0EEFFD0C0EEFFD1C0EEFF9D
:10413000D2C0EEFFD3C0EEFFD4C0EEFFD5C0EEFF7D
:10414000D6C0EEFFD7C0EEFFD8C0EEFFD9C0EEFF5D
:10415000DAC0EEFFDBC0EEFFDCC0EEFFDDC0EEFF3D
:10416000DEC0EEFFDFC0EEFF40D0E0C0EEFFE1C0FA
:10417000EEFFE2C0EEFFE3C0EEFFE4C0EEFFE5C0FD
:10418000EEFFE6C0EEFFE7C0EEFFE8C0EEFFE9C0DD
:10419000EEFFEAC0EEFFEBC0EEFFECC0EEFFEDC0BD
:1041A000EEFFEEC0EEFFEFC0EEFFF0C0EEFFF1C09D
:1041B000EEFFF2C0EEFFF3C0EEFFF4C0EEFFF5C07D
:1041C000EEFFF6C0EEFFF7C0EEFFF8C0EEFFF9C05D
:1041D000EEFFFAC0EEFFFBC0EEFFFCC0EEFFFDC03D
:1041E000EEFFFEC0EEFFFFC0EEFF1CC0EAFF1DC0E9
:1041F000E9FF1200F2B412002E500F0AD8B41200D8
:10420000FF0EE3CF22F0FE0EE3CF23F0FD0EE3CF4F
:1042100024F0FC0EE3CF25F0222A2EA08D8E232A37
:104220002EA28F80242A2EA48F86252A2EA68F8840
:10423000FB0EE3CF26F0FA0EE3CF27F0F90EE3CF23
:1042400028F0F80EE3CF29F0262A8D80272A8D82C8
:10425000282A8D84292A8D865DEC21F0222E33EFC9
:1042600021F02EA08D9E232E38EF21F02EA28F90CC
:10427000242E3DEF21F02EA48F960000252E43EF33
:1042800021F02EA68F980000262E48EF21F08D9069
:104290000000272E4DEF21F08D920000282E52EFC6
:1042A00021F08D940000292E57EF21F08D967FECA0
:1042B00021F02B3E2EEF21F01200D70E2B6E0000C6
:1042C00000000000000075EC21F02B2E5FEF21F0C4
:1042D000D70E2B6E000000000000000075EC21F0EE
:1042E0002B2E6AEF21F000001200000078EF21F081
:1042F0000000000000000000000000001200030E9B
:0C4300002C6E00002C2E81EF21F012002A
:04430C009EB802D085
:10431000FDD7FCD71200D9CFE6FFE1CFD9FFFE0EC3
:10432000DBCFE6FF9AEC1FF0E5520D0EAD6EEEDF2F
:10433000E552E7CFD9FF1200D9CFE6FFE1CFD9FF91
:104340000701D950FD0F506FFF0EDA20516F010E9B
:10435000EA6A5025E96E5151EA22EF50E66E9AEC76
:104360001FF0E55250C7E9FF51C7EAFFEF50E66E74
:104370009AEC1FF0E5520D0EAD6EC8DFE552E7CFA7
:10438000D9FF1200D9CFE6FFE1CFD9FFFD0EDBCF79
:1043900000F0FE0EDBCF01F0026A00C0E6FF01C0B4
:1043A000E6FF02C0E6FF000EE66E070EE66E66EC64
:1043B00024F0F56E050EE15EF550000EE66E070E78
:1043C000E66E7FEC24F0E552E552F3CF54F7F4CFDC
:1043D00055F707015551000AE8AE02D0553505D012
:1043E000500ED8805455000E555503E2500E546FB0
:1043F000556B566B576B57515519E8AE02D0553572
:1044000004D05451565D555157590EE2000E5625B1
:10441000E96E070E5721EA6EEF50AD6E77DF0701A8
:10442000562B000E5723E7D7E552E7CFD9FF1200EE
:10443000D9CFE6FFE1CFD9FF0701526B1A0E525DCB
:1044400011E2FD0EDBCFE9FFDB2AFE0EDBCFEAFF38
:1044500001E3DB2AEF50E66E9AEC1FF0E55207010C
:10446000522BECD70D0EAD6E51DFE552E7CFD9FFE1
:1044700012000701780E506F070E516F0701785137
:104480000701EF6FF06BF151EF1902E1F251F019F2
:1044900018E0070198A502D098950FD0F1C7E6FF64
:1044A0009AEC1FF0E552EFC7E6FF9AEC1FF0E552D9
:1044B0000D0EAD6E2BDF07019895EFC7F1F7F0C732
:1044C000F2F70701F12B000EF223F251000AE8AED9
:1044D00002D0F23505D0FF0ED880F155000EF2550E
:1044E00002E2F16BF26B1200150EE66E3C0EE66E08
:1044F0000FEC24F0E552E552320EE66EB6EC24F0F5
:10450000E5521200D9CFE6FFE1CFD9FFFE0EDBCF97
:1045100053F7E552E7CFD9FF1200D9CFE6FFE1CF3D
:10452000D9FF020EE126FE0EDB507F0BFE0BFD0BCA
:10453000E66E53C7E6FF3BEC24F0E552E5520A0E67
:10454000E66EC6EC24F0E552D4EC24F007EC04F05F
:10455000000901E0FBD78DEC24F0D1EC24F0C4502D
:10456000026E02C003F0026AC35000010210006F25
:1045700003C001F000C0DEFF01C0DDFFDECF00F0B0
:10458000DDCF01F000C0F3FF01C0F4FF00D0D9CFB0
:0A459000E1FFE552E7CFD9FF12006A
:06459A00D9CFE6FFDACFE5
:1045A000E6FFFA0EE3CFD9FFFB0EE3CFDAFFFD0EF5
:1045B000E35209E72D0EDE6EFC0EE31EE32AFD0E2C
:1045C000D8B4E306E31EE652E652E652FD0EE124BD
:1045D000E76EFF0EE220E46EE652F70EE3CFE6FF51
:1045E000F70EE3CFE6FF3DEC23F0F90EE124E96E90
:1045F000FF0EE220EA6E2DEC23F00AE12AEC23F014
:1046000009E12DEC23F008E12AEC23F007E108D0C2
:1046100038EC23F033EC23F038EC23F033EC23F0C8
:1046200038EC23F0DE6AF90EE126FF0EE222FF0EDF
:10463000E3CFDAFFE552FF0EE3CFD9FFE552FC0EE0
:10464000E124E96EFF0EE220EA6EEECFF3FFEFCF3A
:10465000F4FF1200EF380F0B1200EF500F0B02E1C6
:10466000EE52D8841200EF380F0B300FDE6E1200BE
:10467000EE500F0B300FDE6E1200FC0EE3CFE9FFA1
:10468000FD0EE3CFEAFF100EE66EEE6AEE6AEF6A09
:10469000D890FD0EE336FE0EE336ED36ED36EF36FE
:1046A000FF0EE30609E05EEC23F0EE525EEC23F031
:1046B000EE525EEC23F0EDD7E56E1200030EEF2410
:0E46C000E8B6EF6E300EEF24E8BEEF6E000C91
:0246CE001E0EBE
:1046D000F66E080EF76E000EF86E03010900F55035
:1046E0005A6F0900F5505B6F03E15A6701D03DD066
:1046F0000900F550556F0900F550566F0900F55047
:10470000576F09000900F550E96E0900F550EA6E8F
:10471000090009000900F550586F0900F550596F5C
:1047200009000900F6CF5CF3F7CF5DF3F8CF5EF335
:1047300055C3F6FF56C3F7FF57C3F8FF030158539D
:1047400002E1595307E00900F550EE6E5807F8E210
:104750005907F9D75CC3F6FF5DC3F7FF5EC3F8FFE7
:0C47600003015A07000E5B5BBFD712007C
:04476C00D9CFE6FFBC
:10477000E1CFD9FF3F0EC716C66AFE0EDB50C61248
:10478000FC0EDB50C712FD0EDB50030A09E0010AE4
:1047900004E0020A06E1C78C04D0C78CC68801D0A9
:1047A000C688FE0EDB50050A03E0010A04E1928A86
:1047B0009486C79E01D09496949A9488C68AE552AE
:0647C000E7CFD9FF120053
:0A47C600D9CFE6FFE1CFD9FF6C6AFE
:1047D0006B6AFE0EDBB06C88DBA202D06C8C6B8C3B
:1047E000DBB46C8EDBA602D06B8801D06B8ADBA8B1
:1047F00002D06C8401D06C94DBAC02D0A38A01D0CF
:10480000A39ADBAE02D0A38801D0A398FD0EDB50A3
:0E4810006F6E6C8A6B8EE552E7CFD9FF1200F7
:02481E00D9CFF0
:10482000E6FFE1CFD9FFAC6AAB6AFE0EDBB0AC8825
:10483000DBA202D0AC8CAB8CDBB4AC8EDBA602D09E
:10484000AB8801D0AB8ADBA802D0AC8401D0AC9499
:10485000DBAC02D09D8A01D09D9ADBAE02D09D8850
:1048600001D09D98FD0EDB50AF6EAC8AAB8EE55249
:06487000E7CFD9FF1200A2
:0A487600D9CFE6FFE1CFD9FFC26AF7
:10488000C16AC06AFD0EDB407F0B3C0BC26EFE0EA0
:10489000DB500F0B006EFD0EDB38F00B300B001001
:1048A000C16EFE0EDB380F0B070B006EFE0EDB50E9
:1048B000800B0010C06EFD0EDBAE03D09E9C9D8C65
:0C48C000F28CC280E552E7CFD9FF120055
:0448CC00FB0EE3CF2D
:1048D000F6FFFC0EE3CFF7FFFD0EE3CFF8FFFE0E71
:1048E000E3CFE9FFFF0EE3CFEAFFE9CFF3FFEACF23
:1048F000F4FF0900F5CFEFFFEE66FBD71200FE0EC6
:10490000E3CFE9FFFF0EE3CFEAFFF36AF46AEE526A
:0A49100003E0F34AF42AFBD712007B
:06491A00D9CFE6FFE1CF5A
:10492000D9FF020EE126C350DF6E010EC4CFDBFFBC
:10493000DECF00F0DDCF01F000C0F3FF01C0F4FFD7
:0C494000D9CFE1FFE552E7CFD9FF12000C
:04494C0016EE00F073
:1049500026EE00F0F86A3E9CA68EA69C88EC1FF01E
:0C49600067EC23F07EEC1FF0F9D712008A
:04496C00FF0EE35007
:10497000436E480E01D04C0EE76EE72EFED7E76A75
:0C498000E72EFED7432EF7D700001200F0
:04498C00FF0EE350E7
:10499000E84E1200000000D000D000D0E82EFAD778
:0249A000120003
:0649A200C2909D9C120072
:0449A800C2821200B5
:0449AC000200000005
:1049B00001000100000002000100020000000000F0
:1049C00002000100000002000100000002000100DE
:0449D00000000000E3
:0C49D40048656C4C6F2C20576F726C64AF
:1049E0002E000000000000004F682C20506C656114
:1049F00073652E00000000000000000000000000B1
:024A00000000B4
:0E4A02000000010000000000000000000000A5
:104A10000000000000000000010000000000000095
:0A4A2000000000000000000000008C
:020000040030CA
:0E000000FFFEFEFCFFFEFBFFFFFFFFFFFFFF0A
:00000001FF
